:020000040800F2
:1000000000A000205D460008250900082909000815
:100010002D0900083109000835090008000000001A
:100020000000000000000000000000003909000886
:100030003D090008000000004109000845090008CA
:10004000AD460008AD460008AD460008AD460008C4
:10005000AD460008AD460008AD460008AD460008B4
:10006000AD460008AD460008AD460008AD460008A4
:100070004909000855090008AD460008AD460008CA
:10008000610900086D090008AD460008AD4600088A
:1000900079090008AD460008AD460008AD460008E5
:1000A000AD46000885090008AD460008AD460008C9
:1000B000AD460008AD460008AD460008AD46000854
:1000C000AD460008AD460008AD460008AD46000844
:1000D000AD460008AD46000891090008A9090008CE
:1000E000AD460008AD460008AD460008000000001F
:1000F0000000000000000000000000000000000000
:10010000000000000000000000000000AD460008F4
:10011000AD460008AD460008AD46000800000000EE
:10012000AD460008AD460008AD460008AD460008E3
:10013000AD460008000000000000000000000000C4
:10014000AD460008AD4600080000000000000000B9
:10015000000000000000000000000000000000009F
:100160000000000000000000AD460008AD46000899
:10017000AD46000800000000000000000000000084
:0801800000000000AD4600087C
:1001880010B5054C237833B9044B13B10448AFF3C9
:1001980000800123237010BD100000200000000023
:1001A8002447000808B5034B1BB103490348AFF3C4
:1001B800008008BD0000000014000020244700084B
:1001C80010B59CB0002134220FA8CDE90A11CDE961
:1001D8000111CDE90311079100910891022404F05F
:1001E80095FA01224FF480334FF4E01105A8CDE9C8
:1001F8000523CDE90C4309920E9101F049FC08B1A1
:1002080072B6FEE70F220346009268464FF48062FA
:100218002146CDE902320493019401F0CBFF034655
:1002280008B172B6FEE706220FA8CDE912330F9285
:1002380002F030F908B172B6FEE71CB010BD00BF7D
:100248002DE9F04701F0EEFBFFF7BAFF00F06CF87C
:1002580000F002F900F050FA00F06CFA00F0AEF984
:1002680000F0FAF9234B244FDFF89890234E244CE2
:10027800DFF894804FF000629A6004F0D3F904F03C
:100288001FF8388004F022F84AF6CD353B88AB4297
:100298001AD0D4F80038434504D8D4F80038B3F15C
:1002A800005F1BD204F07CF801F0DAFB3368C01A57
:1002B800B0F57A7FEAD920214FF0904002F028FC6F
:1002C80001F0CEFB3060DFE704F018F999F8003050
:1002D800002BDED13B88AB42E4D0DAE72620D4F805
:1002E80004A802F061FED4F8003883F30888D047E8
:1002F800D8E700BF00ED00E0300000202C0000200F
:10030800007000082906002000A00020034B0268A6
:100318009A4200D0704701F097BB00BF002C014003
:1003280072B6FEE7704700BF2DE9F04100248AB09D
:10033800CDE90544CDE90744444B09945969444D36
:1003480041F400215961596901F400210191019991
:10035800596941F480015961596901F48001029198
:100368000299596941F400315961596901F4003120
:1003780003910399596941F4802159615B6903F438
:1003880080230122049370214FF090400126049BA2
:1003980002F0A4FB05A950234FF09040CDE90536A3
:1003A8002027CDE9074402F017FA112305A94FF0D9
:1003B8009040CDE905734FF40048CDE9074402F0B9
:1003C8000BFA05A94FF09040CDE906640894CDF8E2
:1003D800148002F001FA05A928463823CDE90664FD
:1003E80005930326089402F0F7F905A940F2027371
:1003F8004FF090400593069602F0EEF905A92846BD
:100408004FF2C7330593069602F0E6F94FF46043BE
:1004180005A910480593069602F0DEF922464146E2
:100428004FF0904002F05AFB22462846082102F07D
:1004380055FB22462846102102F050FB2246394639
:10044800284602F04BFB0AB0BDE8F08100100240DC
:100458000004004800080048174B00B5586940F0F0
:10046800010058615B6983B0002203F00103114663
:1004780001930C20019B02F039FD0C2002F080FD55
:10048800002211460D2002F031FD0D2002F078FD0A
:1004980000221146102002F029FD102002F070FD04
:1004A80000221120114602F021FD112003B05DF851
:1004B80004EB02F065BD00BF001002400368B3F111
:1004C800804F82B010D00F4A934201D002B07047DB
:1004D8000D4BDA6942F00202DA61DB6903F00203CC
:1004E8000193019B02B0704703F50433DA6942F0C7
:1004F8000102DA61DB6903F001030093009B02B09B
:10050800704700BF000400400010024070B5036847
:1005180088B00024B3F1804FCDE90344CDE9054408
:10052800079404D0224A93422DD008B070BD03F539
:10053800043302255A6942F400325A615A6902F4B6
:1005480000320092009A5A6942F480225A615B692B
:10055800049503F480230193012603A94FF4004373
:100568004FF0904003930796019B02F035F908235A
:100578001048039303A9CDE90454CDE9064602F0D7
:100588002BF908B070BD0C4B0A485A6942F4802216
:100598005A615B6903F4802302240293302503A97E
:1005A800CDE90354029B079402F016F908B070BD18
:1005B80000040040000400480010024000B525482F
:1005C8004FF080420260482200238BB042604FF413
:1005D800FA72CDE90033CDE90233CDE90433CDE930
:1005E8000633CDE90833C0E902320361836100F0C4
:1005F800F1FDF0B90023174800936946029301F012
:100608003FF820BB002260231248059203A9CDE9D8
:100618000332079200F0E8FEB0B90E48042203A99D
:1006280000F0E2FE40B90B48FFF770FF0BB05DF831
:1006380004FBFFF775FEDDE7FFF772FE0548FFF7DD
:1006480065FF0BB05DF804FBFFF76AFEE5E7FFF70F
:1006580067FED7E75C00002000B52548254A026000
:10066800482200238BB042604FF6FF72CDE9003379
:10067800CDE90233CDE90433CDE90633CDE90833BA
:10068800C0E902320361836100F0A4FDF0B90023E0
:10069800174800936946029300F0F2FF20BB00223E
:1006A80060231348059203A9CDE90332079200F0AD
:1006B8009BFEB0B90E48042203A900F095FE40B98C
:1006C8000B48FFF723FF0BB05DF804FBFFF728FE8C
:1006D800DDE7FFF725FE0648FFF718FF0BB05DF8CA
:1006E80004FBFFF71DFEE5E7FFF71AFED7E700BF9B
:1006F800A80000200004004010B50C480C4C002352
:100708004FF4E1310C22C0E90041C0E90233C0E9ED
:100718000432C0E90633C0E9083303F019FC00B914
:1007280010BDBDE81040FFF7FBBD00BF040200206C
:100738000044004010B50C480C4C00234FF4E13144
:100748000C22C0E90041C0E90233C0E90432C0E923
:100758000633C0E9083303F0FBFB00B910BDBDE860
:100768001040FFF7DDBD00BF8C02002000480040AC
:1007780070B503685D4A8AB000249342CDE9054408
:10078800CDE907440546099404D0594A934251D00B
:100798000AB070BD574B584EDA6942F40032DA613C
:1007A800DA6902F400320192019A5A6942F400327D
:1007B8005A615B6903F4003302930C230593029B8F
:1007C800022303224FF09040069305A90723CDE9A1
:1007D800082302F001F8494A1023C6E900233046ED
:1007E8008023C6E90243C6E90444C6E9064402F088
:1007F800A5F9002870D1424C42492E670023802277
:100808002046C4E90013C4E90232C4E90433C4E948
:100818000633756202F092F900285AD10022114677
:100828006C672620656202F061FB262002F0A8FBB7
:100838000AB070BD2F4B344EDA69344842F4802236
:10084800DA61DA6902F480220392039A5A6942F45F
:1008580080225A615B6903F4802304934FF4406358
:100868000593049B022306934FF0030C072305A965
:10087800CDE908C301F0B0FF254A80233046C6E918
:100888000024C6E90243C6E90444C6E9064402F066
:1008980055F920BB1F4C20496E6710220023C4E97C
:1008A800001220468022C4E90232C4E90433C4E9B4
:1008B8000633756202F042F9A0B9002211462720DA
:1008C8002C67656202F012FB272002F059FB0AB080
:1008D80070BDFFF725FDA1E7FFF722FD8BE7FFF7C6
:1008E8001FFDD7E7FFF71CFDE7E700BF0044004006
:1008F80000480040001002403801002080000240FB
:10090800F40000206C0002407C0100200004004834
:1009180030000240C00100201C000240FEE700BF7A
:10092800FEE700BFFEE700BFFEE700BFFEE700BF2F
:10093800704700BF704700BF704700BF704700BFD7
:10094800014802F069BA00BFC0010020014802F066
:1009580063BA00BF7C010020014802F05DBA00BF05
:10096800F4000020014802F057BA00BF3801002007
:10097800014800F041BF00BF34000020014800F0EA
:100988007FBA00BF1403002008B5044802F00EFE29
:10099800BDE80840014803F0B9BC00BF04020020CC
:1009A800014802F003BE00BF8C0200200A4B9A697E
:1009B80042F001029A619A6982B002F00102009243
:1009C800009ADA6942F08052DA61DB6903F08053F9
:1009D8000193019B02B07047001002401F4B70B595
:1009E8009A691F4C42F400629A619B6988B003F4CB
:1009F800006301A90293064603A8029B01F018FDB3
:100A080001F0FEFC174A1849A2FB00239B0C013B8E
:100A18000022C4E90013204640F2E7332261A260B5
:100A2800A261E36000F034FB054610B1284608B027
:100A380070BD204600F0BEF905460028F6D1192001
:100A480002F09EFA0F2E01D90125EFE72A4631461A
:100A5800192002F04BFA054B1E60E7E70010024030
:100A68001403002083DE1B43002C014004000020F7
:100A7800026A036A23F48033036230B44468436D26
:100A88000D6823F4803323F070032B438D6822F420
:100A9800003242EA05420D4DA8420BD005F5A0559B
:100AA800A84207D005F58065A84203D005F5806502
:100AB800A84204D14D6924F4803444EA05244968E5
:100AC8004460436530BC816502627047002C014078
:100AD800026A036A23F48013036230B44468436DE6
:100AE8000D6823F0807323F4E04343EA05238D68FF
:100AF80022F4001242EA05520D4DA8420BD005F52A
:100B0800A055A84207D005F58065A84203D005F591
:100B18008065A84204D14D6924F4802444EA8524E0
:100B280049684460436530BCC1650262704700BFD4
:100B3800002C01402DE9F041066A036A0F6823F092
:100B480001030362D0F80480836923F4803323F01F
:100B580073031F438B6826F002061E433C4B9842E2
:100B680004460D462ED003F5A05398420FD003F546
:100B7800806398420BD003F58063984207D06B6876
:100B8800C4F80480A76163632662BDE8F081EB685E
:100B980043B3082B4AD12F4B26F00C069C4246F053
:100BA800080624D1AB6933F400732CD16B6933F494
:100BB800807231D1AA6928F4407848EA020848EAE4
:100BC8000308DCE7CB6873B3082B3BD0224841F617
:100BD8009231FFF7A7FBEB6826F008061E4326F0C4
:100BE8000406DFE726F00C061A4B9C42DAD003F520
:100BF80080639C42D6D003F580639C42BFD1AB6929
:100C080033F40073D2D0144841F69F31FFF78AFBC2
:100C18006B6933F48072CDD00F484FF4DD51FFF784
:100C280081FB6B69C6E726F00C06BBE70A4841F66C
:100C38009231FFF777FBEB6826F008061E4326F093
:100C48000406D1E726F00C0646F00806AAE700BF1E
:100C5800002C0140004001403C4700082DE9F041CC
:100C6800066A036A0F6823F480730362D0F804806D
:100C7800C36923F4803323F073031F438B6826F47E
:100C8800007646EA0326254B984204460D4620D0B6
:100C9800234B984206D0234B9C4203D003F5806334
:100CA8009C420ED1AB6933F4007326D16B6933F4DF
:100CB80080722BD1AA6928F4405848EA021848EAF9
:100CC80003186B68C4F80480E761E3632662BDE833
:100CD800F081CB6833F0080205D0134841F62B4168
:100CE800FFF720FBEB6826F4006646EA0326AB69AB
:100CF80033F4007326F48066D8D00B4841F63941A6
:100D0800FFF710FB6B6933F48072D3D0064841F6C5
:100D18003A41FFF707FB6B69CCE700BF002C0140A5
:100D280000400140004401403C470008F0B5056A16
:100D3800036A0E6823F4805303624268C36923F090
:100D4800807323F4E64343EA06268B6825F40055AE
:100D580045EA0335144B984283B004460F460BD03E
:100D680003F5A053984207D003F58063984203D057
:100D780003F58063984207D17B6933F480710AD107
:100D880022F4804242EA83127B686260E66123644F
:100D9800256203B0F0BD0548019241F67B41FFF79B
:100DA800C1FA7B69019AEBE7002C01403C47000837
:100DB800704700BF2A4A0368934210B504461FD003
:100DC800B3F1804F1CD0A2F59432934218D002F5AB
:100DD8008062934214D002F50062934210D002F56B
:100DE800983293420CD002F58062934208D002F503
:100DF8008062934204D01B4840F2D711FFF792FA61
:100E080094F83D30012B1ED122681549022384F83D
:100E18003D30D3688A4243F00103D36015D0B2F164
:100E2800804F12D0104B9A420FD003F580639A423C
:100E38000BD003F59C339A4207D0136843F00103A3
:100E48000020136010BD012010BD9168074B0B40B6
:100E5800062B02D0B3F5803FEFD1002010BD00BFB4
:100E6800002C01403C470008000400400700010036
:100E7800704700BF704700BF704700BF704700BF92
:100E8800036870B5DE681C69A107054601D5B2077D
:100E980054D4620701D573073DD4200701D5310723
:100EA80027D4E30601D5F00610D4E10701D5F207EF
:100EB80062D4230652D5300666D4600601D5710681
:100EC80073D4A20601D5B3064DD470BD2B686FF05C
:100ED80010021A6108222A77DB6913F4407F28463A
:100EE80074D1FFF7C5FF2846FFF7C6FF00232B770D
:100EF800DBE72B686FF008021A6104222A77DB69A6
:100F08009A0728465FD1FFF7B3FF2846FFF7B4FFDB
:100F180000232B77C5E72B686FF004021A610222C1
:100F28002A779B6913F4407F284649D1FFF7A0FF31
:100F38002846FFF7A1FF00232B77AEE76FF00202E8
:100F48001A61012202779B69990736D1FFF790FF52
:100F58002846FFF791FF00232B779AE7E205ACD5E7
:100F680033061AD4A9E72B686FF0200228461A61C5
:100F7800BDE8704000F020BC2B686FF001021A61D8
:100F88002846FFF7C3F994E72B686FF080021A61CF
:100F9800284600F013FCE1058FD52B686FF48072AA
:100FA8001A61284600F00CFC87E72B686FF04002B6
:100FB8001A612846FFF762FF83E7FFF75BFFCAE77E
:100FC800FFF758FFB7E7FFF755FFA1E7FFF752FF15
:100FD8008CE700BF2D4A0368904230B43CD0B0F192
:100FE800804F1DD0A2F59432904219D002F580624C
:100FF800904215D002F59C32904241D002F58062B1
:1010080090423DD002F58062904239D04D698C689B
:101018000A6823F080032B430360C462826210E0F5
:101028004A68CC6823F07003134323F440734A6979
:10103800234323F080038C6813430A680360C46267
:101048008262012343610369DB0703D5036923F047
:101058000103036130BC70474C68CA6823F0700311
:10106800234323F4407313434A6923F08003134353
:1010780003608B68C3620B6883620B690363E0E7F4
:10108800CC684A6923F440732343EEE7002C0140FF
:10109800002800F0998003684C4A934210B5044632
:1010A8001FD0B3F1804F1CD0A2F59432934218D0D0
:1010B80002F58062934214D002F50062934210D088
:1010C80002F5983293420CD002F58062934208D020
:1010D80002F58062934204D03D484FF48D71FFF7CA
:1010E80021F9A36833F010020AD023F04002202A25
:1010F80006D0402B04D0364840F21B11FFF712F9F6
:10110800236933F4807236D12368B3F1804FE368E2
:101118003ED04FF6FE72013B93423BD8A36933F0B1
:10112800800340D194F83D3003F0FF02002B45D0F6
:101138002146022384F83D3051F8040BFFF74AFF9B
:10114800012384F8483084F83E3084F83F3084F82E
:10115800403084F8413084F8423084F8433084F8D1
:10116800443084F8453084F8463084F8473084F8B1
:101178003D30002010BDB3F5007FC5D014484FF4B2
:101188008E71FFF7CFF82368B3F1804FE368C0D1C1
:10119800002BC3D10E4840F21D11FFF7C3F8A36915
:1011A80033F08003BED00A484FF48F71FFF7BAF8C6
:1011B80094F83D3003F0FF02002BB9D184F83C20AD
:1011C8002046FFF7F5FDB3E701207047002C0140EA
:1011D8003C470008002800F0998003684C4A934275
:1011E80010B504461FD0B3F1804F1CD0A2F594323D
:1011F800934218D002F58062934214D002F500623F
:10120800934210D002F5983293420CD002F58062D6
:10121800934208D002F58062934204D03D4840F2E0
:101228003951FFF77FF8A36833F010020AD023F092
:101238004002202A06D0402B04D0364840F23A51CA
:10124800FFF770F8236933F4807236D12368B3F15D
:10125800804FE3683ED04FF6FE72013B93423BD885
:10126800A36933F0800340D194F83D3003F0FF02C6
:10127800002B45D02146022384F83D3051F8040B59
:10128800FFF7A8FE012384F8483084F83E3084F83C
:101298003F3084F8403084F8413084F8423084F894
:1012A800433084F8443084F8453084F8463084F874
:1012B800473084F83D30002010BDB3F5007FC5D01D
:1012C800144840F23B51FFF72DF82368B3F1804FE3
:1012D800E368C0D1002BC3D10E4840F23C51FFF760
:1012E80021F8A36933F08003BED00A4840F23D518B
:1012F800FFF718F894F83D3003F0FF02002BB9D13E
:1013080084F83C202046FFF7D9F8B3E7012070475E
:10131800002C01403C4700082DE9F041066A036AA9
:101328000F6823F010030362D0F80480836923F068
:10133800807323F4E64343EA07278B6826F02006E8
:1013480046EA0316244B984204460D4620D0234B08
:10135800984206D0224B9C4203D003F580639C42FE
:101368000ED1AB6933F4007326D16B6933F4807204
:101378002BD1AA6928F4406848EA820848EA830819
:101388006B68C4F80480A761A3632662BDE8F08196
:10139800CB6833F0080205D0124841F6DE31FEF77B
:1013A800C1FFEB6826F0800646EA0316AB6933F402
:1013B800007326F04006D8D00A4841F6EB31FEF714
:1013C800B1FF6B6933F48072D3D0064841F6EC3133
:1013D800FEF7A8FF6B69CCE7002C014000400140F4
:1013E800004401403C470008142A70B516460546DB
:1013F8000C464AD93C2A4CD1236823F0100223F426
:10140800803323F01003602B07D0994B9A4204D005
:10141800984841F2C301FEF785FFA36833F0020341
:1014280004D0944841F2C401FEF77CFF236933F0ED
:10143800040304D08F4841F2C501FEF773FF95F805
:101448003C30012B00F01281012385F83C30142E2A
:1014580016D8DFE816F08500150015001500B8004D
:10146800150015001500E4001500150015004100D1
:101478001500150015006900150015001500240059
:101488000120002385F83C3070BD7B4BD340DB073F
:10149800B2D4784841F2C201FEF744FFACE72868AD
:1014A800764B984205D0734841F22711FEF73AFF70
:1014B80028682146FFF70CFB2B682069596D41F419
:1014C80000615965596D21F4806159655A6D42EA88
:1014D80000225A650020D4E72868684B984210D04B
:1014E800B0F1804F0DD0A3F59433984209D003F59D
:1014F8008063984205D05F4841F20211FEF712FF5F
:1015080028682146FFF712FC2B682069D96941F445
:101518000061D961D96921F48061D961DA6942EA47
:101528000022DA610020ACE72868544B984205D0C5
:10153800504841F21411FEF7F5FE28682146FFF7DE
:1015480097FA2B682069596D41F008015965596D62
:1015580021F0040159655A6D02435A65002090E74D
:101568002868464B98421CD0B0F1804F19D0A3F59B
:101578009433984215D003F58063984211D003F54F
:101588009C3398420DD003F58063984209D003F547
:101598008063984205D0374841F2CF01FEF7C2FE7A
:1015A80028682146FFF7C6FA2B682069996941F037
:1015B80008019961996921F0040199619A690243C6
:1015C8009A6100205DE728682C4B984214D0B0F14E
:1015D800804F11D0A3F5943398420DD003F5806362
:1015E800984209D003F59C33984205D021484FF41E
:1015F8008751FEF797FE28682146FFF78DFE2B6876
:101608002069996941F400619961996921F48061BF
:1016180099619A6942EA00229A61002031E72868B4
:10162800164B984210D0B0F1804F0DD0A3F59433EB
:10163800984209D003F58063984205D00D4841F2DD
:10164800F101FEF76FFE28682146FFF707FB2B68BC
:101658002069D96941F00801D961D96921F00401EB
:10166800D961DA690243DA6100200AE7022070BD15
:10167800400001003C47000811111100002C0140F6
:101688004A4A036893422DE9F04104460D4617D0B3
:10169800B3F1804F14D0A2F59432934210D002F5E2
:1016A800806293420CD002F50062934208D002F5A2
:1016B8009832934204D03E4840F2AC71FEF732FEB5
:1016C8002B6833F0300306D0402B04D0384840F262
:1016D800AD71FEF727FEAB6833F080034FD194F865
:1016E8003C30012B54D02368DFF8C080012102224E
:1016F80084F83C1084F83D2043455E689F681FD0FD
:101708002A6826F0700616435E60B3F1804F0AD04F
:10171800284A934207D002F58062934203D002F52B
:101728009C32934204D1AA6827F0800717439F6030
:101738000020012384F83D3084F83C00BDE8F081A6
:101748006A6832F4401126D0B1F5800F23D0B1F584
:10175800000F20D0B1F5400F1DD0154840F2C171DF
:10176800FEF7E0FD26F470026E682B68324322F023
:1017780070021A43236843455A60D4D0C5E70C4821
:1017880040F2AE71FEF7CEFD94F83C30012BAAD1A1
:101798000220BDE8F08126F4700616432A6826F078
:1017A80070061643014A5660BDE700BF002C014091
:1017B8007447000800040040704700BF704700BF2E
:1017C800704700BF704700BF704700BF704700BF39
:1017D800704700BF704700BF704700BF704700BF29
:1017E800704700BF704700BF704700BF704700BF19
:1017F800704700BF704700BF2DE9F84F03685C6968
:10180800D3F804809F68D3F80CB0D3F810A0D3F8AD
:10181800189014F00106054620D017F001060DD0E7
:1018280001229A60BB0700F1C4807E0700F1E380C3
:1018380017F0080600F0E8804FF48056F8050BD53D
:101848002B684FF48072B9059A6000F1AE807A0572
:1018580040F1CC8046F40056F80365D4270702D53A
:101868001BF0100F6BD1600703D51BF0080F40F079
:101878008D80A10704D52B68DB689A0740F0828029
:10188800630602D51AF0100F48D1A70602D51AF040
:10189800080F62D1E00603D52B681B6999077CD134
:1018A800A20302D518F0100F5ED1E30302D518F099
:1018B800080F60D1270405D518F0040F06D12B684E
:1018C80004225A60002E40D1BDE8F88FE00504D507
:1018D80019F0010F18BF46F00106A10504D519F04B
:1018E800020F18BF46F00206620504D519F0040F6E
:1018F80018BF46F004062305E1D519F07009DED0BB
:10190800B9F1400F00F08B8057D8B9F1200F78D08B
:10191800B9F1300F5FD146F0200656E02B6810224F
:1019280046F480661A61B0E72B684FF48032B90339
:101938009A6036D47A0354D546F400468EE72B686D
:10194800102246F40076DA608DE76B6A1E4328465B
:101958006E62FFF74FFFBDE8F88F2B6808221A6107
:101968002846FFF741FF95E72B6810225A60284662
:10197800FFF73CFF99E72B6808225A602846FFF7D3
:1019880037FF97E72846FFF729FF79E72B680822F2
:10199800DA602846FFF724FF6BE72846FFF722FFA7
:1019A8007EE72846FFF712FF58E72846FFF70CFFA7
:1019B80052E7FFF707FF002640E7B9F1500F1DD0A7
:1019C800B9F1600F08BF46F480762B689A6922F057
:1019D80070029A6174E7B9F1100FF6D146F0080663
:1019E800F3E73B0317D546F4803637E73B050ED5BA
:1019F80046F4804630E74FF400661FE746F080065D
:101A0800E3E746F01006E0E7FFF7E2FE16E72846B0
:101A1800FFF7E0FE20E72846FFF7DEFE1EE746F068
:101A28004006D2E7074A08B5136843F0100313606D
:101A3800032001F03DFA0F20FEF7D0FFFEF7B6FFB6
:101A4800002008BD00200240034A044B11681B789F
:101A58000B441360704700BF6003002000000020A3
:101A6800014B1868704700BF6003002038B5044672
:101A7800FFF7F6FF631C054602D0044B1B781C4495
:101A8800FFF7EEFF431BA342FAD338BD0000002046
:101A9800002800F063832DE9F043036883B004460F
:101AA800002B00F0B180190700F04A82DA0748D508
:101AB800636833F4803203D0B3F5A02F40F022825C
:101AC800B44A536803F00C03042B24D0536803F082
:101AD8000C03082B1CD06368B3F5803F00F0EC8141
:101AE800002B00F03482B3F5A02F00F0FA82A94B46
:101AF8001A6822F480321A601A6822F480221A6066
:101B0800A44AA168D36A23F00F030B43D362DEE132
:101B18005368DB03DFD54FF4003393FAA3F29D4AF1
:101B2800116893FAA3F3B3FA83F303F01F030122B6
:101B380002FA03F30B4203D06368002B00F0E8813C
:101B480023689F072FD52369012B00F268816369F9
:101B58001F2B00F26D818F4B5A6812F00C0F40F06A
:101B68002181022393FAA3F28A4A116893FAA3F314
:101B7800B3FA83F303F01F03012202FA03F30B42C3
:101B880003D02369934240F0C3818248F822016858
:101B980092FAA2F26369B2FA82F2934021F0F80253
:101BA8001343036023681D072ED5A369012B00F298
:101BB8006C81002B40F04281012696FAA6F1764A04
:101BC800744FB1FA81F10A4492004FF00208136091
:101BD800FFF746FF054605E0FFF742FF401B0228D6
:101BE80000F2AA8198FAA8F398FAA8F398FAA8F349
:101BF8007A6A98FAA8F3B3FA83F303F01F0306FA94
:101C080003F31342E8D12368580736D5E368012B5C
:101C180006D9052B04D061484FF4FA71FEF782FB10
:101C28005C4BDA69D10000F13A81DA6942F08052FE
:101C3800DA61DB6903F080530193019B4FF00108DF
:101C4800574D2B68DA0540F16781E368012B00F0F6
:101C5800FA81002B00F0A481052B4E4B1A6A00F084
:101C68004D8222F001021A621A6A22F004021A62F4
:101C7800EEE1B8F1000F40F02E82E069022800F290
:101C88001181002800F08180424D6B6803F00C033D
:101C9800082B00F00F82022840F03882236A33F4C0
:101CA800803304D03D4840F24121FEF73BFB636A94
:101CB80033F4402223F4802110D0B2F5801F0DD0D8
:101CC800B2F5001F0AD0B1F5401F07D0B3F5601F69
:101CD80004D0324840F24221FEF724FB4FF08073D3
:101CE80093FAA3F3B3FA83F303F1845303F584134C
:101CF8009B0000221A60FFF7B3FE264E05464FF000
:101D08000078012705E0FFF7ABFE401B022800F230
:101D1800138198FAA8F3326898FAA8F3B3FA83F310
:101D280003F01F0307FA03F31342ECD1D4E90813B5
:101D380072680B4322F47412134373604FF080737C
:101D480093FAA3F3B3FA83F303F1845303F58413EB
:101D58009B00104D1F60FFF783FE4FF0007704468D
:101D6800012605E0FFF77CFE001B022800F2E48054
:101D780097FAA7F32A6897FAA7F3B3FA83F303F05D
:101D88001F0306FA03F31342ECD0002003B0BDE8AA
:101D9800F08300BF0010024020819010AC4700087B
:101DA800007000405A6802F00C02082A00F07681A0
:101DB8002269002A00F02181012595FAA5F3B3FADA
:101DC80083F303F1845303F584139B00B64F1D601E
:101DD800FFF746FE4FF00208064605E0FFF740FE13
:101DE800801B022800F2A88098FAA8F33A6898FAAB
:101DF800A8F3B3FA83F303F01F0305FA03F31342BE
:101E0800ECD03968F82292FAA2F26369B2FA82F247
:101E1800934021F0F80213433B602368C3E6A348CC
:101E280040F28711FEF77EFA63691F2B7FF693AEA7
:101E38009E484FF4C471FEF775FA8CE6012595FAB1
:101E4800A5F29B4B984FB2FA82F213449B004FF0D5
:101E580002081D60FFF704FE064604E0FFF700FED7
:101E6800801B022868D898FAA8F398FAA8F398FA79
:101E7800A8F37A6A98FAA8F3B3FA83F303F01F0376
:101E880005FA03F31342E9D0BDE688484FF4E4713C
:101E9800FEF748FAA369002B3FF48EAECEE74FF069
:101EA8000008CDE681484FF40E71FEF73BFAE06971
:101EB80000287FF4E9AE68E77B4A136843F480336F
:101EC8001360D36AA16823F00F030B43D362FFF7B3
:101ED800C7FD754F05464FF40038012604E0FFF7AB
:101EE800BFFD401B642827D898FAA8F33A6898FAE7
:101EF800A8F3B3FA83F303F01F0306FA03F31342BC
:101F0800EDD01DE6694840F24F11FEF70BFAD7E510
:101F1800012003B0BDE8F0832B6843F480732B6085
:101F2800FFF79EFD06462B68DB053FF58EAEFFF7F3
:101F380097FD801B6428F6D9032003B0BDE8F08321
:101F48005A4840F24911FEF7EDF92368AEE5564DBF
:101F58002B6823F480332B602B6823F480232B60B9
:101F6800EB6AA26823F00F031343EB62FFF778FDD7
:101F78004FF400380646012704E0FFF771FD801B87
:101F88006428D9D898FAA8F32A6898FAA8F3B3FA73
:101F980083F303F01F0307FA03F31342EDD1CFE5F0
:101FA800414D2B6A23F001032B622B6A23F00403B3
:101FB8002B62FFF755FD4FF002090646012714E092
:101FC80099FAA9F36A6A99FAA9F3B3FA83F303F0C1
:101FD8001F0307FA03F313423FF44BAEFFF740FD2C
:101FE80041F28833801B9842A6D899FAA9F399FA46
:101FF800A9F3002BE4D02A6AE5E7012696FAA6F3AE
:10200800B3FA83F303F1845303F584139B00264F3B
:102018001A60FFF725FD4FF00208054604E0FFF7B8
:102028001FFD401B022887D898FAA8F33A6898FA47
:10203800A8F3B3FA83F303F01F0306FA03F313427A
:10204800EDD12368AFE5184A136A43F00103136220
:10205800FFF706FD144F05464FF00209012615E06B
:1020680099FAA9F37A6A99FAA9F3B3FA83F303F010
:102078001F0306FA03F313427FF4FBADFFF7F0FCEE
:1020880041F28833401B98423FF656AF99FAA9F3BC
:1020980099FAA9F3002BE3D03A6AE4E75B68DE0318
:1020A8003FF586AE5DE500BF00100240AC47000872
:1020B8002081901001283FF469AE6B68226A03F40E
:1020C800803191427FF424AF606A03F47013181AC8
:1020D80018BF01205AE6224AD36923F08053D361FE
:1020E800CBE503F18043A3F53C331A6842F4802220
:1020F8001A601A6842F480321A6001E542F004025C
:102108001A621A6A42F001021A62A1E74FF080735C
:1021180093FAA3F3B3FA83F303F1845303F5841317
:102128009B0000221A60FFF79BFC4FF000770446E3
:10213800012605E0FFF794FC001B02283FF6FCAEE1
:1021480097FAA7F32A6897FAA7F3B3FA83F303F089
:102158001F0306FA03F31342ECD116E60120704779
:10216800001002400E4A536803F00C01082901D000
:102178000C487047C3F3834010B4D26A0A4C0B4929
:10218800205C5DF8044BDB034CBF064B084B02F0A8
:102198000F028A5C48BFB3FBF2F303FB00F0704701
:1021A8000010024000127A00E4470008F4470008D3
:1021B80000093D00002800F0E28003682DE9F041A5
:1021C8001E070D46044600F0D480022D00F2CB8095
:1021D800794A136803F00703AB420CD2136823F063
:1021E80007032B431360136803F00703AB4202D0C5
:1021F8000120BDE8F081236898071ED5A16831F059
:10220800800214D021F02002902A10D021F0400240
:10221800A02A0CD021F01002C02A08D0F02906D03C
:1022280040F2D9216548FEF77DF8A1682368644823
:10223800426822F0F0020A434260D90733D5636846
:10224800022B00F2B080012B00F09B80022B0CBF08
:102258004FF00072022292FAA2F15949086892FAE4
:10226800A2F2B2FA82F202F01F02012101FA02F28E
:102278000242BDD0524E726822F0030213437360CB
:10228800FFF7EEFB41F28838074605E0FFF7E8FB69
:10229800C01B404500F28E807368626803F00C032F
:1022A800B3EB820FF2D1444A136803F00703AB4241
:1022B80009D9136823F007032B431360136803F04D
:1022C8000703AB4294D123685A0718D5E16831F463
:1022D80080620ED021F40072B2F5A06F09D0B1F57A
:1022E800C06F06D04FF447713448FEF71BF8E16819
:1022F80023683348426822F4E0620A4342601B07BD
:1023080018D5226932F480630DD022F40073B3F536
:10231800A06F08D0B2F5C06F05D0284840F223312D
:10232800FEF700F8226926494B6823F4605343EA14
:10233800C2034B60FFF716FF214BF0225B6892FA4D
:10234800A2F2B2FA82F203F0F003D3401D4A1E490A
:10235800D35C1E4A20FA03F308681360FEF73EFBBD
:102368000020BDE8F081154840F2C221FDF7DAFFF0
:102378002EE7124840F2C121FDF7D4FF25E70120DE
:1023880070474FF4003292FAA2F10D49096892FAA7
:10239800A2F2B2FA82F202F01F0203FA02F20A4231
:1023A8007FF468AF24E705484FF43871FDF7BAFFAA
:1023B800636848E703201CE700200240AC47000898
:1023C8000010024094490008040000200800002082
:1023D800084B4FF4E0625B6892FAA2F2B2FA82F21A
:1023E80003F4E06304490548D3400068CB5CD84057
:1023F800704700BF00100240A449000808000020F0
:10240800084B4FF460525B6892FAA2F2B2FA82F279
:1024180003F4605304490548D3400068CB5CD840B6
:10242800704700BF00100240A449000808000020BF
:1024380038B50D460446D0B105B3134B13490F22E6
:1024480022605A6802F0030262605A6802F0F002E1
:10245800A2605A6802F4E062E2605B68DB0803F499
:10246800E06323610B6803F007032B6038BD08485D
:1024780040F28541FDF756FF002DDED1044840F2B9
:102488008641FDF74FFFD8E70010024000200240C8
:10249800AC4700082DE9F0439E4A0368934283B095
:1024A800044600F23181D8034ED5636833F4407393
:1024B80040F05581984BDA69D10000F13581DA692D
:1024C800964E42F08052DA61DB6903F08053019343
:1024D800019B3368DA054FF0010540F12C81DFF8E4
:1024E8003882D8F8203013F4407320D0616801F4A2
:1024F80040729A421CD0D8F820104FF4803321F44F
:10250800407093FAA3F2864FB2FA82F23A449200EC
:102518000126166093FAA3F3B3FA83F33B449B00B6
:102528000022CF071A60C8F8200000F12B816168EB
:10253800794A136A23F440730B4313621DB1D369BC
:1025480023F08053D3612368DD0709D5A1680329E7
:1025580000F20A817048026B22F003020A43026308
:1025680098070FD5E16831F4403205D0C7216D488E
:10257800FDF7D8FEE16823686748026B22F4403211
:102588000A43026359070FD5216931F4402205D067
:10259800D3216448FDF7C6FE216923685E48026BB3
:1025A80022F440220A4302639A060FD5E16931F00A
:1025B800100205D0DE215B48FDF7B4FEE16923680F
:1025C8005548026B22F010020A4302639F030AD5A2
:1025D800216B31F4800240F0CE804F48426822F4EB
:1025E80080020A4342605E0610D5216A31F020025B
:1025F80006D04FF480714B48FDF794FE216A23689A
:102608004548026B22F020020A4302631D0710D5D9
:10261800616931F4401206D040F221114148FDF7BA
:1026280081FE616923683C48026B22F440120A4328
:102638000263D80610D5A16931F4400206D040F2F1
:102648002B113848FDF76EFEA16923683248026BEA
:1026580022F440020A430263990510D5A16A31F4B5
:10266800000206D040F23B112E48FDF75BFEA16A3E
:1026780023682948426822F400020A4342601A0685
:1026880027D5616A31F480721DD021F02002B2F59D
:10269800887F18D021F04002B2F5907F13D021F046
:1026A8001002B2F5A07F0ED0B1F5B87F0BD021F0A3
:1026B8003002B2F5C07F06D040F25B111948FDF731
:1026C80031FE616A23681448C26A22F4F8720A4328
:1026D800C26213F4805313D0E26A32F4807305D0D7
:1026E80010484FF4C671FDF71DFEE26A0A490B6BEC
:1026F80023F48073002013430B6303B0BDE8F08319
:10270800184603B0BDE8F08306487021FDF70AFEBD
:102718002368C8E6FF120300001002400070004062
:102728000081901004480008294E3368DA054FF0FC
:1027380000053FF5D4AE336843F480733360FFF788
:102748008FF907463368DB053FF5C9AEFFF788F90F
:10275800C01B6428F6D9032003B0BDE8F0831D48E8
:102768007621FDF7DFFDA5E6BC211A48FDF7DAFD65
:10277800A1682368EEE6EC211648FDF7D3FD216B2E
:1027880023682AE7FFF76CF94FF00209074615E0BE
:1027980099FAA9F3D8F8242099FAA9F3B3FA83F39C
:1027A80003F01F0306FA03F313427FF4C0AEFFF7EA
:1027B80057F941F28833C01B9842CCD899FAA9F34B
:1027C80099FAA9F3002BE3D0D8F82020E4E700BF5A
:1027D80000700040044800082DE9F04FB0F1904F18
:1027E80085B00646884616D0B54B984213D003F5F7
:1027F800806398420FD003F5806398420BD003F5AD
:102808008063984207D003F58063984203D0AD48AF
:10281800B221FDF787FDD8F800108BB223B10B0C5D
:102828001B04002B00F02E81A648B321FDF77AFD8A
:10283800D8F80430012B18D9A3F11102012A14D9B0
:102848009A1E012A11D923F40012B2F5881F0CD060
:10285800B3F5041F09D0B2F5901F06D0B3F5081FD1
:1028680003D09848B421FDF75DFDD8F80010002981
:1028780000F0CE80DFF85CB2DFF85C92002401251E
:10288800A54015EA010300F0BE80D8F8040000F066
:1028980003014F1E012F40F2BE804FEA440A03276E
:1028A80007FA0AF7FF4303294DD0D8F80850022D3C
:1028B80000F2DD80F26805FA0AF502EA070C45EA3B
:1028C8000C050229F5603ED1B6F1904F17D07C4A2D
:1028D800964214D07C498E4211D001F580618E4217
:1028E8000DD001F580618E4209D001F580618E42DC
:1028F80005D074480193E221FDF714FD019BD8F837
:1029080010000C280BD9A0F10E01012907D96D4838
:102918000193E321FDF706FDD8F81000019BE508B7
:1029280006EB850504F007012A6A89004FF00F0EAF
:1029380088400EFA01F122EA01010143D8F80400A7
:10294800296200F00301356801FA0AF12F40394382
:1029580010F4403F316054D0DBF8185045F00105C1
:10296800CBF81850DBF8185024F0030101F180412E
:1029780005F0010501F58031039504F0030C039D72
:102988008F684FEA8C0C0F2505FA0CF5B6F1904FBD
:1029980027EA050513D04A4A964200F084804A4F38
:1029A800BE4200F08680494FBE4276D0484FBE42B4
:1029B8000CBF0427052707FA0CFC45EA0C058D60B7
:1029C800D9F80810DD43C70254BF29401943C9F894
:1029D8000810D9F80C10820254BF29401943C9F8CD
:1029E8000C10D9F80410870354BF29401943C9F8BB
:1029F8000410D9F80010C20354BF29401943C9F87C
:102A08000010D8F80010013431FA04F37FF437AF1E
:102A180005B0BDE8F08FD8F80C20012A0DD9032A9B
:102A28000BD028480193C321FDF77CFCD8F804009B
:102A3800D8F80C20019B00F00301B7684FEA440A5C
:102A48004FF0030E0EFA0AFE02FA0AFC27EA0E07F6
:102A58004CEA0707B760726822EA050CC0F3001554
:102A6800A54045EA0C056FEA0E0775601BE7154897
:102A78000193D421FDF756FCD8E90105019B00F02C
:102A8800030117E7D8F80430012B7FF6F3AEA3F162
:102A98001102012A3FF6D4AEE7E6032707FA0CFC39
:102AA80045EA0C058BE7012707FA0CFC45EA0C05FB
:102AB80085E7022707FA0CFC45EA0C057FE700BF0B
:102AC800000400483C48000800080048000C004882
:102AD80000100048001002400004014070B506468E
:102AE80015460C4659B1012D02D835B9B46270BDEE
:102AF800064840F2A511FDF715FCB46170BD034806
:102B08004FF4D271FDF70EFCEDE700BF3C4800081A
:102B180038B505460C4641B1696904EA010324EA5F
:102B2800010444EA0344AC6138BD03484FF4DE7144
:102B3800FDF7F8FBF0E700BF3C480008002800F06C
:102B4800B88003685C4A934210B5044625D0143215
:102B5800934222D0143293421FD0143293421CD095
:102B68001432934219D01432934216D0143293423D
:102B780013D002F5627293420FD0143293420CD0F4
:102B88001432934209D01432934206D0143293423D
:102B980003D04A489321FDF7C5FB636833F0100260
:102BA8005DD1A36833F0400364D1E36833F0800358
:102BB80068D1236933F4807202D0B3F5007F66D1FF
:102BC800636933F4806202D0B3F5006F68D1A369FA
:102BD80033F0200303D039489921FDF7A3FBE069BE
:102BE80030F4405304D035489A21FDF79BFBE06947
:102BF8002168D4E901321343E2681343226913437D
:102C080062694FF0020C1343A26984F821C0134390
:102C18000A6822F47F5222F030021343284A034301
:102C280091420B600FD9274B274A0B44A2FB032381
:102C38001B09264A9B00C4E90F234FF48073002028
:102C48002384A06310BD224B1F4A0B44A2FB03231D
:102C58001B09204A03FA0CF3C4E90F23EDE7B3F587
:102C6800804F9ED015489421FDF75CFBA36833F094
:102C780040039AD011489521FDF754FBE36833F0DF
:102C8800800396D00D489621FDF74CFB91E70B4841
:102C98009721FDF747FB636933F4806297D093E788
:102CA80006489821FDF73EFBA36933F0200396D030
:102CB80091E70120704700BF0800024074480008EF
:102CC80007040240F8FBFDBFCDCCCCCC0004024089
:102CD800F8FFFDBF000002402DE9F0415D1E1E46D1
:102CE8004FF6FE739D4204460F46904635D894F839
:102CF8002030012B3AD0012384F8203094F8213079
:102D0800012B05D0002384F820300220BDE8F08193
:102D1800022284F8212025680022A2632A6822F072
:102D280001022A60226C9340E26B536063686E6014
:102D3800102BE36A0BBFC5F80880AF60EF60C5F8D9
:102D48000C80B3B12B6843F00E032B602B6843F063
:102D5800010300202B60BDE8F0810A484FF4A671FA
:102D6800FDF7E0FA94F82030012BC4D10220BDE829
:102D7800F0812B6843F00A032B602B6823F00403CF
:102D88002B60E3E77448000808B390F82120022A72
:102D9800034606D004210022816380F82020012008
:102DA80070470268116821F00E0110B4046CC06B02
:102DB8001160116821F0010111600122A2404FF455
:102DC80080714260198400205DF8044B704701202F
:102DD800704700BF90F82120022A03D004228263A2
:102DE800012070470268116821F00E0110B5C46B0C
:102DF8001160116821F001011160026C01219140FC
:102E0800426B61604FF4807CA0F820C012B19047FB
:102E1800002010BD104610BD70B4C66B026C31683E
:102E28000468042393400B4225680ED015F0040F64
:102E38000BD02268920603D4226822F00402226092
:102E4800C26A7360CAB170BC1047022393400B4238
:102E580015D015F0020F12D02268920606D4226807
:102E680022F00A022260012280F82120826A73601F
:102E7800002180F82010002AE5D170BC7047082393
:102E880093400B42F9D02B07F7D52368016B23F049
:102E98000E032360012303FA02F24FF48074726078
:102EA800048483630029E8D070BC0847806B7047AE
:102EB800C31E042B10B504460ED80A4A2302D46850
:102EC8004FF6FF0103F4E0630C40234343F0BF6374
:102ED80043F40033D36010BD0348AB21FDF722FA59
:102EE800EBE700BF00ED00E0AC4800080F2A70B522
:102EF800164605460C4637D80F2C30D81D4BDB68D4
:102F0800C3F30223C3F10700042803F1040228BF16
:102F18000420062A18D9033B4FF0FF329A4026EACC
:102F280002064FF0FF31814024EA01049C40002D45
:102F380044EA06040BDB05F16045240105F561450B
:102F4800E4B285F8004370BD00263346E9E70A4B32
:102F580005F00F0524012B44E4B21C7670BD074828
:102F6800C421FDF7DFF9C9E70448C321FDF7DAF901
:102F7800C2E700BF00ED00E0FCEC00E0AC48000850
:102F8800002809DB4109064A00F01F00012303FA63
:102F980000F042F8210070470248D721FDF7C2B976
:102FA80000E100E0AC48000800280EDB43090949AD
:102FB8000122203300F01F0002FA00F041F823003C
:102FC800BFF34F8FBFF36F8F70470348E721FDF7BB
:102FD800A9B900BF00E100E0AC480008BFF34F8F7B
:102FE8000549064BCA6802F4E0621343CB60BFF39D
:102FF8004F8F00BFFDE700BF00ED00E00400FA05B9
:103008000C4BDB6813F0100305D00B49CA6942F07A
:1030180002021023CA61074AD268520706D5064938
:10302800CA6942F0010243F00403CA61014AD3604D
:10303800704700BF0020024068030020064B186953
:1030480010F0800006D00549054A59605A60186991
:10305800C0F3C010704700BF00200240230167453D
:10306800AB89EFCD034A136943F080030020136155
:10307800704700BF0020024070B50446FEF7F0FC20
:10308800104D064601E0631C10D1EB68D807FAD44E
:10309800EB68990644BF2023EB600A4BDA68D20636
:1030A8000CD4D86810F0040008D170BD24B1FEF724
:1030B800D7FC801BA042E8D9032070BDFFF7A0FF12
:1030C800012070BD002002402DE9F84F354F1D4604
:1030D8003B7E012B63D001233B76431E022B064621
:1030E8008A4690464ED8BAF1006F0AD32E4BB3F8F1
:1030F800CC30B3F5807F4AD0802B4CD02B4B9A45EF
:1031080003D92B48B121FDF70DF94CF25030FFF7E8
:10311800B3FF98BB012E03D0022E0CBF0226042653
:103128000024DFF898B00AEB4606A146C4F1200354
:10313800C7F81C90A4F1200228FA04F005FA03F35A
:10314800184325FA02F2DBF8103010431FFA80FC0E
:1031580043F00103CBF810304CF25030AAF800C00D
:10316800FFF78AFFDBF8103023F001030AF1020AA7
:103178001034CBF8103008B9B245D7D100233B76CC
:10318800BDE8F88F0A48B021FDF7CCF8ABE7094B4A
:103198009A45B6D8B9E7084B9A45B2D8B5E70220A0
:1031A800BDE8F88F6803002000F7FF1FFFFF000845
:1031B800E4480008FFFF0308FFFF01080020024061
:1031C8002DE9F843554E337E012B00F0A3800123EF
:1031D80033760368012B8146884605D95048A621D5
:1031E800FDF7A0F8D9F80030012B6BD0D9F80430DE
:1031F800B3F1006F0AD34B4AB2F8CC20B2F5807F06
:1032080050D0802A7AD0484A93420DD94448BC21EC
:10321800FDF788F8434BB3F8CC30B3F5807F6AD01C
:10322800802BD9F804306CD0D9F8082003EBC223DE
:103238003D4A013B934240D84CF25030FFF71CFF07
:10324800074668BB4FF0FF33C8F80030D9E901538F
:1032580005EBC3239D4223D2344C07E0D9E9013260
:1032680005F5006503EBC223AB4215D9F761236965
:1032780043F0020323616561236943F0400323613E
:103288004CF25030FFF7F8FE236923F00203236164
:103298000028E3D0C8F8005000233376BDE8F8834F
:1032A8000120F9E7224A9342B0D8D9F8082003EB65
:1032B800C2231F4A013B9342BED91948BD21FDF7DD
:1032C80031F8B9E74CF25030FFF7D6FE0028E7D1C5
:1032D800164CF061236943F004032361236943F02A
:1032E800400323614CF25030FFF7C6FE236923F0F8
:1032F80004032361D0E7D9F80430D6E70D4A934296
:1033080084D8D9F8082003EBC2230A4A013B934228
:1033180092D9D2E70220BDE8F88300BF68030020F5
:103328001C49000800F7FF1FFFFF000800200240AB
:10333800FFFF0308FFFF0108026852E8003F23F47B
:10334800907342E800310029F7D102F1080353E8ED
:10335800003F23F0010302F1080C4CE8003100297A
:10336800F3D1036E012B06D000232022C0F8802061
:1033780083660366704752E8003F23F0100342E873
:1033880000310029F0D052E8003F23F0100342E852
:1033980000310029EFD1E7E770B5C56F202D2DD199
:1033A80051B34AB30023A0F852200446C164C0F8C0
:1033B8008430A0F85020006F2126E66760B1134ED4
:1033C8004363134622688662114EC662114E066335
:1033D8002832FFF781FC98B922684023136202F172
:1033E800080353E8003F43F0800302F1080141E875
:1033F80000300028F3D170BD012070BD022070BDDF
:103408001023C4F884300120E56770BDE13400085A
:10341800293500084135000838B50368044653E8E3
:10342800002F22F4907243E800210029F7D103F11C
:10343800080252E8002F22F0010203F1080040E8D8
:1034480000210029F3D1226E012A26D09968490665
:103458001A460ED400230F21A4F85A30116291693C
:10346800202541F0080191611846C4F88050236670
:1034780038BD03F1080252E8002F22F0400203F1A0
:10348800080040E800210029F3D1606FB0B1416322
:10349800FFF77AFCA0B92268DCE753E8002F22F096
:1034A800100243E800210029D0D053E8002F22F071
:1034B800100243E800210029EFD1C7E71A46C9E7FF
:1034C800606FFFF7F3FC2028E5D11023C4F884309F
:1034D800032038BD704700BF08B58369406A202BB8
:1034E80018D000230268A0F8523002F1080353E80C
:1034F800003F23F0800302F1080040E80031002972
:10350800F3D152E8003F43F0400342E8003100297C
:10351800F7D108BDFFF7DEFF08BD00BF704700BF49
:1035280008B5406AFFF7FAFF08BD00BF704700BF43
:10353800704700BF704700BF406A0268C16F10B58E
:10354800D0F8804093681B0601D521290DD09368D7
:103558005B0601D5222C16D0D0F8843043F0100336
:10356800C0F88430FFF7E6FF10BD0023A0F8523002
:1035780052E8003F23F0C00342E800310029F7D1A8
:103588002023C367E3E70023A0F85A30FFF7D4FEEF
:10359800E2E700BF08B5406A0023A0F85A30A0F857
:1035A8005230FFF7C7FF08BD704700BF0368DA69EC
:1035B800196840F60F0C12EA0C0F2DE9F0419D68CE
:1035C80004467FD1970602D58E0600F1F780206E5B
:1035D800012824D0D00202D56F0200F1F48016062B
:1035E80014D4500601D54A0601D4BDE8F08153E849
:1035F800002F22F0400243E800210029F7D12023C0
:10360800E367E1662046FFF765FFEEE70D06E8D5BC
:10361800E36E002BE9D02046BDE8F0411847D706F5
:10362800D8D5CE06D6D510221A629A68550640F12A
:10363800DD80606F0268526892B2002AD5D0B4F873
:1036480058109142D1D9A4F85A208269202A2FD043
:1036580053E8002F22F4807243E800210029F7D1B3
:1036680003F1080252E8002F22F0010203F10805D5
:1036780045E800210029F3D103F1080252E8002FA0
:1036880022F0400203F1080545E800210029F3D1A2
:103698002022C4F88020216653E8002F22F010026F
:1036A80043E800210029F7D1FFF76EFBB4F8581062
:1036B80002236366B4F85A30C91A204689B2FFF764
:1036C80073FF92E7674805F00106084030433FF46E
:1036D8007EAFD5071F4609D5C80507D50120186252
:1036E800D4F8840040F00100C4F88400950760D540
:1036F8008EB102201862D4F8840040F00400C4F8A7
:103708008400500707D504201862D4F8840040F0DC
:103718000200C4F8840010070BD501F020003043E4
:1037280007D008201862D4F8840040F00800C4F8D4
:10373800840016050AD54D0108D54FF400601862BB
:10374800D4F8843043F02003C4F88430D4F88430AB
:10375800002B3FF44AAF900601D589063FD4D4F830
:103768008450BB6805F0280503F040031D4320463C
:1037780073D0FFF7E1FD23689A6852062BD503F151
:10378800080252E8002F22F0400203F1080040E846
:1037980000210029F3D1606FE8B1334B4363FFF791
:1037A80019FB00283FF421AF606FBDE8F041436B7F
:1037B80018475507AFD5002EA5D1ACE7836E002B6F
:1037C8007FF42AAF11E74FF4801220461A62BDE851
:1037D800F04100F091BC2046FFF7ACFE05E7A36E70
:1037E800002BBCD0204698472768B8E7B4F85A1091
:1037F800B4F85A2092B289B2002A3FF4F6AEB4F86F
:103808005820511A89B200293FF4EFAE53E8002F2F
:1038180022F4907243E800200028F7D103F108024F
:1038280052E8002F22F0010203F1080545E80020C4
:103838000028F3D12022C4F88020A066206653E82F
:10384800002F22F0100243E800200028F7D10223BD
:1038580063662046FFF7A8FEC7E6FFF76BFEC4F8CD
:103868008450C2E6200100049D350008406A08B56E
:1038780001234366036E012B02D0FFF759FE08BDF2
:10388800B0F858104908FFF78FFE08BD08B58369DE
:10389800406A202B29D000220368A0F85A2053E858
:1038A800002F22F4807243E800210029F7D103F1A8
:1038B800080252E8002F22F0010203F1080C4CE83C
:1038C80000210029F3D103F1080252E8002F22F069
:1038D800400203F1080C4CE800210029F3D1202212
:1038E800C0F88020026E012A07D000234366036EC9
:1038F800012B13D0FFF71AFE08BD53E8002F22F062
:10390800100243E800210029EFD053E8002F22F0ED
:10391800100243E800210029EFD1E6E7B0F858107B
:10392800FFF742FE08BD00BF38B54268A54B9A4272
:10393800044600F2A780A36833F4805304D0A24859
:1039480040F63A31FCF7EEFCE36833F4405304D018
:103958009D4840F63B31FCF7E5FC236A33F40063ED
:1039680004D0994840F63C31FCF7DCFC236933F479
:10397800806203D0B3F5C06F40F09880636933F07C
:103988000C0246D1002B44D0A36933F4407304D011
:103998008D484FF43461FCF7C5FCE16931F400430C
:1039A80005D040F641318848FCF7BCFCE169226843
:1039B8002569A36810682B43656920F4164020F038
:1039C8000C002B4303430B4313605368E068256ADC
:1039D80023F44053034353609068A36920F4306094
:1039E8002B43034379489360824251D0784B9A42E3
:1039F80015D0784B9A4200F0B580774B9A4200F088
:103A0800C680764B9A4275D00023C4E91A33012048
:103A180038BD6D4840F63F31FCF784FCB4E703F548
:103A2800E6331B6B03F44033B3F5003F75D00FD872
:103A3800002B68D0B3F5803FE6D1B1F5004F72D0C6
:103A4800FEF790FB60B90023C4E91A33002038BDA3
:103A5800B3F5403FD8D1B1F5004F00F0E28060489F
:103A680063684FF6EF7200EB5300B0FBF3F3A3F17A
:103A780010019142C8D82268D3600023C4E91A33E0
:103A8800002038BD504840F63931FCF74BFC52E76E
:103A9800544B1B6B03F00303013B022B0CD9B1F50C
:103AA800004F00F08980FEF7ABFCCBE7464840F6B4
:103AB8003E31FCF737FC61E74B4AB1F5004FD35C68
:103AC80000F09480082B9FD801A252F823F000BF81
:103AD800153B0008AF3A0008673A0008113A000899
:103AE800493A0008113A0008113A0008113A00084A
:103AF800293B00083B4B1B6B03F44003B3F5000F55
:103B08000BD02AD82BB9B1F5004F58D0FEF760FC7E
:103B180098E7B3F5800F90D076E7B1F5004F7DD0E8
:103B28004FF400409CE7FEF71DFB00288BD04300B4
:103B380062684FF6EF7103EB5203B3FBF2F3A3F1A4
:103B480010028A423FF660AF23F00F02216892B25A
:103B5800C3F342031343CB6075E7B3F5400F3FF45B
:103B68007AAF51E703F5E4331B6B03F44023B3F555
:103B7800002FD2D006D8002BC5D0B3F5802F3FF444
:103B88005CAF41E7B3F5402F3FF465AF3CE703F581
:103B9800E2331B6B03F44013B3F5001FBDD006D806
:103BA800002BB0D0B3F5801F3FF447AF2CE7B3F537
:103BB800401F3FF450AF27E7FEF722FCB5E7FEF7BA
:103BC80007FCB2E740548900584900080038014012
:103BD8000044004000480040004C004000500040B5
:103BE80000127A000010024090490008082B3FF6A6
:103BF8000BAF01A252F823F0C73B0008C13B0008F5
:103C08002B3C0008113A00082F3B0008113A000825
:103C1800113A0008113A0008253C00084FF4803397
:103C280086E7014B84E700BF0024F400436AFF2BBA
:103C380010B5044600F295801A070AD5616B31F475
:103C4800004240F09D802068426822F400420A4306
:103C58004260D8070AD5A16A31F4003240F0988052
:103C68002068426822F400320A43426099070AD564
:103C7800E16A31F4803240F093802068426822F48F
:103C880080320A4342605A070AD5216B31F48022F8
:103C980040F08E802068426822F480220A43426005
:103CA800D8060AD5A16B31F4805240F0898020688B
:103CB800826822F480520A438260990609D5E16B32
:103CC80031F4005254D12068826822F400520A4329
:103CD80082605A062BD52368464A93420CD0A2F537
:103CE8007442934208D002F58062934204D042485D
:103CF80040F6F131FCF716FB236C5BB3B3F5801F7C
:103D080066D12268536843F480135360606C30F4C2
:103D1800C00306D0384840F6F731FCF703FB606C67
:103D280022685168636A21F4C001014351601B068F
:103D38000FD5A26C32F4002305D02F4840F6FF318E
:103D4800FCF7F0FAA26C21684B6823F400231343B4
:103D58004B6010BD2168636A4A6822F480124A6089
:103D6800E5E7254840F6C231FCF7DCFA636A63E709
:103D780040F6EA312048FCF7D5FAE16B636AA2E71E
:103D880040F6C7311C48FCF7CDFA616B636A5AE705
:103D980040F6CE311848FCF7C5FAD4E909315FE797
:103DA80040F6D5311448FCF7BDFAE16A636A64E766
:103DB80040F6DC311048FCF7B5FA216B636A69E715
:103DC80040F6E3310C48FCF7ADFAA16B636A6EE785
:103DD80040F6F2310848FCF7A5FA2268216C5368CE
:103DE80023F480130B43B1F5801F53608ED0636AB0
:103DF8009DE700BF00380140584900082DE9F84305
:103E0800089F0D46804601681646994601E0781CD1
:103E18000CD1CC6935EA04030CBF4FF0010C4FF00C
:103E2800000CB445F3D00020BDE8F883FDF718FE78
:103E3800A0EB0900B8421DD8E7B1D8F800100B680C
:103E48005A07E6D5802DE4D0402DE2D0CC6914F095
:103E5800080411D1CB691B05DBD54FF400630B6255
:103E68004046FFF769FA2023C8F8843088F878407C
:103E78000320D9E70320D7E7082440460C62FFF760
:103E88005BFA0023C8F8844088F878300120CBE733
:103E980070B50446002682B0C0F88460FDF7E0FDE6
:103EA80023681A68120705460ED41B685B0726D4D8
:103EB80000232022E26784F87830C4F8802018466E
:103EC8002366636602B070BD6FF07E43009332468E
:103ED80003464FF400112046FFF790FF236800289F
:103EE800E3D053E8002F22F0800243E800210029A4
:103EF800F7D12023E36784F878100320E2E76FF016
:103F08007E43009300222B464FF480012046FFF7A2
:103F180075FF0028CCD0236853E8002F22F4907254
:103F280043E800210029F7D103F1080252E8002FE5
:103F380022F0010203F1080040E800210029F3D132
:103F48002023C4F8803084F878100320BAE700BF33
:103F580000285ED0836910B50446002B33D003686F
:103F68002D4A93420CD0A2F57442934208D002F530
:103F78008062934204D029484FF49671FCF7D2F935
:103F8800E36F002B3FD02268616A2423E36713683C
:103F980023F00103136091BB2046FFF7C5FC0128FD
:103FA8002BD023685A6822F490425A609A6822F00B
:103FB8002A029A601A6842F0010220461A60BDE897
:103FC8001040FFF765BF0368134A9342D8D0A2F5A3
:103FD80074429342D4D002F580629342D0D002F565
:103FE80080629342CCD002F580629342C8D00B48DD
:103FF80040F23111FCF796F9C2E7012010BD2046C6
:10400800FFF714FEC8E784F878302046FCF7B0FBC9
:10401800B9E70120704700BF00380140584900083F
:1040280038B5044600232220C4F88430C4F8800040
:10403800606F6165A4F8582070B125684363134622
:104048000A4605F124011B4D85621B4DC5621B4DB7
:104058000563FEF741FE28BB23694BB1236853E88B
:10406800002F42F4807243E800210029F7D100E0D4
:10407800236803F1080252E8002F42F0010203F11D
:10408800080040E800210029F3D103F1080252E8B2
:10409800002F42F0400203F1080141E80020002807
:1040A800F3D138BD10222023C4F884200120C4F89D
:1040B800803038BD9538000875380008413500084B
:1040C800D0F88030202B15D101B10AB901207047F2
:1040D80030B400230468036663681B0207D554E8FC
:1040E800003F43F0806344E80035002DF7D130BC31
:1040F800FFF796BF02207047704700BF034AD2F807
:10410800883043F47003C2F88830704700ED00E04F
:1041180099B130B4FF220A4D0A4C00EB010C11464C
:1041280010F8013B53406045EA5C82EA0102E15C19
:10413800F6D142EA012030BC70474FF6FF70704755
:10414800AC490008AC4A0008B0F1000C70B541DB7E
:104158000025234CA4FB0C031846DB0802F1FF3EA4
:1041680003EB830322B1ACEB430330334B550135EA
:104178005FEAD00C5FFA8EF2ECD101F805C00B783B
:104188002D2B02D101354FF0010CBCEB650F4FEA26
:1041980065021DDA0CF1FF3EA5EB0C034C1E8E44A4
:1041A8000B4414441EF8012F13F8010D0244D2B237
:1041B8008EF8002093F800C0A2EB0C0018709EF84F
:1041C80000008444ACEB0202A6458EF80020E9D139
:1041D800084670BD2D23CCF1000C0B700125B8E703
:1041E800CDCCCCCC2DE9F041804684B00F461546A5
:1041F80072B6FEF723FF1D4B1D4E3422DA6033687A
:10420800E3B1112B1AD035B3013DADB2BC1E07EB9B
:104218004505A8EB070701E0AC421CD034F8022F93
:10422800002339190120FEF74FFF0028F4D0FEF7CC
:1042380019FF62B6022004B0BDE8F0810023012412
:10424800694601A8CDE90033CDF808800394FEF74C
:10425800B7FF3460D7E7FEF705FF62B6336803207F
:104268000133336004B0BDE8F08100BF0020024094
:104278008803002030B585B072B6FEF7DFFE0E4B1E
:104288000E4D3422DA6001240023694601A8CDE9E5
:10429800013503940093FEF793FF0F22002329466C
:1042A8002046FEF711FF0446FEF7DCFE62B6B4FABC
:1042B80084F0400905B030BD0020024000600008CD
:1042C800014B188880B27047006000080C4A0D48FE
:1042D800538982B09BB2ADF80430918989B2ADF8A8
:1042E800041003EB01430360D38907499BB2ADF87F
:1042F8000430128A03EB02430B6002B0704700BF20
:1043080000680008900300208C030020204B98428E
:1043180000D070470368DA69D20610B5044600D4A5
:1043280010BD10221A62FFF777F8636F19491A68EF
:104338000B785268FE2B10D04B79152B1ED04FF4FA
:1043480080720021134800F0E1F9BDE810401149DE
:104358000F484FF48072FFF7B3BE0B79CC2BEBD12B
:104368000D4B93F800010028E6D1C2F5807218467B
:1043780000F0BEF9012280F80021E0E78B791A2BC2
:10438800DDD1CB79032BDAD1044B01221A70D6E7A1
:104398000402002094030020280500209C0400202B
:1043A800384BDA6F202A00D070471B68DA6952064A
:1043B800FAD5DB691B06F7D570B5334B1C7886B088
:1043C8001CB9324B1B68012B01D906B070BD304EA9
:1043D800FDF746FB3368C01AB0F5FA7FF5D9FDF74B
:1043E8003FFBB0F5FA6FF0D9FDF73AFB294D306085
:1043F800214680222846CDE90044CDE90244CDE992
:10440800044400F083F9244B244C1868FE232B70D5
:104418001A236B7103230C226946EB8001232B724C
:10442800FFF792FE1E4B0C220DEB02011868FFF7F6
:104438008BFE6A4603CA03ABC5F80900C5F80D1020
:1044480003CB1288A5F81120C5F839001A88C5F8D9
:104458003D10532359212846A5F841206B70FFF7DA
:1044680057FEA5F85900FDF7FBFA2060FDF7F8FAAA
:1044780023689842FAD0074902485B22FEF78CFF6E
:10448800A3E700BF040200209C0400209804002039
:1044980024050020A004002090030020200500200F
:1044A8008C03002038B5124D124CA871FE2241F23F
:1044B800CC532A60AB800B78EB71487828720122C4
:1044C80004230A2128466A726B70FFF721FE68816F
:1044D800FDF7C6FA2060FDF7C3FA23689842FAD0C0
:1044E800BDE83840024904480C22FEF755BF00BF1A
:1044F800A00400202005002004020020F0B5434C51
:10450800617883B020460831FFF702FE002301934B
:1045180020B1002384F8003103B0F0BD3C4BDA6FC2
:10452800202AF6D11B68DA695206F2D5DB691B0628
:10453800EFD56579C92D0ED0CA2D36D0C82D19D022
:10454800324800214FF4807284F8001103B0BDE8AE
:10455800F04000F0DBB8E2792E4EA37903EB02239A
:10456800326893422DD09A42EAD9A11D2846FFF716
:1045780099FFE5E7D4F8062027490192A2F1011333
:10458800A3F538438B42DBD8224D2B68012B01D988
:10459800FEF724FD002601A9C8200196FFF782FF37
:1045A8001E4A012316602B60CAE71D4E3378002B84
:1045B800C6D1FFF75FFE307018BB3220FDF756FA00
:1045C800BEE7164F62783868023A02EBD27200F101
:1045D8000060C2F34F0200F5F04004F10801FFF754
:1045E80001FE03280190ABD1336862780133336050
:1045F8003B68023B13442846A11D3B60FFF752FF6E
:104608009EE701A92846FFF74DFFD6E728050020B9
:104618000402002098040020FECF0100940400202A
:104628002906002010B5094C09492068036843F0A1
:10463800100303604FF480722046FFF741FD2268A3
:10464800936843F00103936010BD00BF040200208B
:1046580094030020DFF834D0FFF750FD0C480D49D3
:104668000D4A002302E0D458C4500433C4188C42C5
:10467800F9D30A4A0A4C002301E013600432A2422B
:10468800FBD300F011F8FBF7DBFDFEE700A00020EC
:10469800000000200C000020B44B0008100000208F
:1046A8002C060020FEE7000070B50D4D0D4C641B74
:1046B800A4100026A64209D10B4D0C4C00F02EF890
:1046C800641BA4100026A64205D170BD55F8043B12
:1046D80098470136EEE755F8043B98470136F2E76C
:1046E800AC4B0008AC4B0008AC4B0008B04B0008C2
:1046F8000A44914200F1FF3300D1704710B511F818
:10470800014B03F8014F9142F9D110BD0244034611
:10471800934200D1704703F8011BF9E7F8B500BFD1
:10472800F8BC08BC9E467047F8B500BFF8BC08BC8A
:044738009E467047E2
:10473C00447269766572732F53544D333246337815
:10474C00785F48414C5F4472697665722F5372638F
:10475C002F73746D3332663378785F68616C5F7475
:10476C00696D2E6300000000447269766572732FC8
:10477C0053544D3332463378785F48414C5F447222
:10478C00697665722F5372632F73746D333266338F
:10479C0078785F68616C5F74696D5F65782E630013
:1047AC00447269766572732F53544D3332463378A5
:1047BC00785F48414C5F4472697665722F5372631F
:1047CC002F73746D3332663378785F68616C5F7207
:1047DC0063632E630000000002030405060708094A
:1047EC000A0B0C0D0E0F101001020304050607082E
:1047FC00090A0B0C0D0E0F10447269766572732F3B
:10480C0053544D3332463378785F48414C5F447291
:10481C00697665722F5372632F73746D33326633FE
:10482C0078785F68616C5F7263635F65782E630094
:10483C00447269766572732F53544D333246337814
:10484C00785F48414C5F4472697665722F5372638E
:10485C002F73746D3332663378785F68616C5F6781
:10486C0070696F2E63000000447269766572732F55
:10487C0053544D3332463378785F48414C5F447221
:10488C00697665722F5372632F73746D333266338E
:10489C0078785F68616C5F646D612E630000000066
:1048AC00447269766572732F53544D3332463378A4
:1048BC00785F48414C5F4472697665722F5372631E
:1048CC002F73746D3332663378785F68616C5F6315
:1048DC006F727465782E6300447269766572732FFB
:1048EC0053544D3332463378785F48414C5F4472B1
:1048FC00697665722F5372632F73746D333266331E
:10490C0078785F68616C5F666C6173682E63000019
:10491C00447269766572732F53544D333246337833
:10492C00785F48414C5F4472697665722F537263AD
:10493C002F73746D3332663378785F68616C5F66A1
:10494C006C6173685F65782E630000004472697651
:10495C006572732F53544D3332463378785F484128
:10496C004C5F4472697665722F5372632F73746D4A
:10497C003332663378785F68616C5F756172742E60
:10498C0063000000040802000000000000000000AA
:10499C0001020304060708090000000001020304D9
:1049AC0000C1814001C0804101C0804100C18140F3
:1049BC0001C0804100C1814000C1814001C08041E3
:1049CC0001C0804100C1814000C1814001C08041D3
:1049DC0000C1814001C0804101C0804100C18140C3
:1049EC0001C0804100C1814000C1814001C08041B3
:1049FC0000C1814001C0804101C0804100C18140A3
:104A0C0000C1814001C0804101C0804100C1814092
:104A1C0001C0804100C1814000C1814001C0804182
:104A2C0001C0804100C1814000C1814001C0804172
:104A3C0000C1814001C0804101C0804100C1814062
:104A4C0000C1814001C0804101C0804100C1814052
:104A5C0001C0804100C1814000C1814001C0804142
:104A6C0000C1814001C0804101C0804100C1814032
:104A7C0001C0804100C1814000C1814001C0804122
:104A8C0001C0804100C1814000C1814001C0804112
:104A9C0000C1814001C0804101C0804100C1814002
:104AAC0000C0C101C30302C2C60607C705C5C404C2
:104ABC00CC0C0DCD0FCFCE0E0ACACB0BC90908C832
:104ACC00D81819D91BDBDA1A1EDEDF1FDD1D1CDC22
:104ADC0014D4D515D71716D6D21213D311D1D01092
:104AEC00F03031F133F3F23236F6F737F53534F482
:104AFC003CFCFD3DFF3F3EFEFA3A3BFB39F9F838F2
:104B0C0028E8E929EB2B2AEAEE2E2FEF2DEDEC2CE1
:104B1C00E42425E527E7E62622E2E323E12120E051
:104B2C00A06061A163A3A26266A6A767A56564A441
:104B3C006CACAD6DAF6F6EAEAA6A6BAB69A9A868B1
:104B4C0078B8B979BB7B7ABABE7E7FBF7DBDBC7CA1
:104B5C00B47475B577B7B67672B2B373B17170B011
:104B6C005090915193535292965657975595945401
:104B7C009C5C5D9D5F9F9E5E5A9A9B5B9959589871
:104B8C00884849894B8B8A4A4E8E8F4F8D4D4C8C61
:104B9C0044848545874746868242438341818040D1
:044BAC00AD0100084F
:044BB000890100086F
:0C4BB400010000001000000000127A0058
:040000050800465D4C
:00000001FF
